:1000000000308A00472800000000A70104302702C2
:10001000031826282708A000A00DA00DA00DF83079
:10002000A0052008A1001F08C73921049F00000077
:1000300000000000000000002230270784001F1588
:100040001F1920281E088000A70A06286E28060807
:10005000A6006F28A7012830270203184628FF3082
:100060006600061C2F280310A60CA50CA40CA30CDC
:10007000A20C03183D2805123E280516EF30650036
:10008000FF30660006184028A70A2B287028840134
:1000900083019F308400073080008130840080130A
:1000A000A001A01D5B280730810181308400000879
:1000B000C0390F3880006400813084000008C039E6
:1000C000200480009F30840080011F083839C13827
:1000D0009F00FF30660006186928052827282A286F
:0400E0006928630028
:02400E00F33F7E
:00000001FF
